:020000040000FA
:06000000F3EF06F0120010
:06080000F3EF06F0120008
:06082A000100040E0000B5
:0808300000020000200000009E
:08083800D9CFE6FFE1CFD9FFA3
:10084000040EE126DE6ADE6ADE6ADD6ADD52DD5212
:10085000FB0EDBCF00F0FC0EDBCF01F0FD0EDBCF9B
:1008600002F0FE0EDBCF03F0D9CFE9FFDACFEAFFCB
:10087000030EEB500318E8AE02D0033408D000504A
:10088000EE5C0150EE580250EE580350EE580FE265
:100890000C0EE66ED3EC06F0E552D9CFE9FFDACFC5
:1008A000EAFFEE2A000EEE22EE22EE22D1D7040E4F
:1008B000E15C02E2E16AE552E16EE552E7CFD9FF81
:1008C00012000F0EC16E070EB46E936A300E926E58
:1008D0000F0E946EF19E1200D9CFE6FFE1CFD9FF43
:1008E000020EE1268250020B01E0010E080DF3CF4B
:1008F00002F08250010B040DF3CF01F08050200B69
:1009000001E0010EE824006E8050100B01E0010EA2
:10091000002401240224DE6EDD6ADECF00F0DDCF8C
:1009200001F000C0F3FF01C0F4FF020EE15C03E23E
:1009300000D0E16AE552E16EE552E7CFD9FF12003F
:100940008092010EE66EE66AE66AE66A75DFE552B7
:10095000E552E552E5528084010EE66EE66AE66AEB
:10096000E66A6ADFE552E552E552E5528094010EEF
:10097000E66EE66AE66AE66A5FDFE552E552E55250
:10098000E55212008082010EE66EE66AE66AE66AC9
:1009900053DFE552E552E552E5528084010EE66EE2
:1009A000E66AE66AE66A48DFE552E552E552E55254
:1009B0008094010EE66EE66AE66AE66A3DDFE5527D
:1009C000E552E552E5521200380E816EB9DF320E63
:1009D000E66EE66AE66AE66A2FDFE552E552E55220
:1009E000E552010E816EACDF320EE66EE66AE66A13
:1009F000E66A22DFE552E552E552E5520D0E816EC0
:100A00009FDF320EE66EE66AE66AE66A15DFE552B9
:100A1000E552E552E552060E816E92DF320EE66E29
:100A2000E66AE66AE66A08DFE552E552E552E55213
:100A30001200010E816E84DF0A0EE66EE66AE66A37
:100A4000E66AFADEE552E552E552E5521200D9CFE8
:100A5000E6FFE1CFD9FF020E816E72DF0A0EE66E6D
:100A6000E66AE66AE66AE8DEE552E552E552E552F4
:100A7000FD0EDBCFE6FFFE0EDB50280DF350E552F6
:100A8000E724E76EFE0EE7CFDBFFFD0EDB6AFE0E0E
:100A9000DB50F36EFD0EDBCFF4FFF350F45C10E29D
:100AA000140E816E4DDF010EE66EE66AE66AE66AB6
:100AB000C3DEE552E552E552E552FD0EDB2AE7D7EB
:100AC000E552E7CFD9FF1200D9CFE6FFE1CFD9FF3A
:100AD000FE0EDB50816E56DF010EE66EE66AE66AB8
:100AE000E66AAADEE552E552E552E552E552E7CF65
:100AF000D9FF1200D9CFE6FFE1CFD9FFFD0EDBCF42
:100B0000E9FFFE0EDBCFEAFFEF500EE0FD0EDBCF7C
:100B1000E9FFDB2AFE0EDBCFEAFF01E3DB2AEF5021
:100B2000E66ED2DFE552EAD7E552E7CFD9FF1200F1
:100B30000201246B300E926EF00E936EEF0E206F5A
:100B400020C281FF040E216F2151000825E22051AF
:100B5000FE0BE842206F20C281FF050EE66EE66ABA
:100B6000E66AE66A69DEE552E552E552E5528150F1
:100B7000100B09E08150200B06E08150400B03E090
:100B80008150800B01E10AD80201240502E12551C0
:100B900004D02105216FD8D7CBD71200F00E936E69
:100BA00081CF23F202012315226F0F0E2015206F33
:100BB00020512211206F81CF23F2F00E2315226FD6
:100BC000F00E225D01E0F7D7936A06D826C225F21F
:100BD0000201010E246F12000201276B100E275D27
:100BE00014E22751EA6A000FE96E020EEA22EF5082
:100BF000205D08E12751EA6A100FE96E020EEA2231
:100C0000EFCF26F22729276FE9D726C281FF640E8E
:100C1000E66EE66AE66AE66A0FDEE552E552E552FE
:100C2000E55212000201286B070E285D1DE280DFED
:100C30000201296F2851EA6A2A0FE96E020EEA22A0
:100C400029C2EFFF2851EA6A2A0FE96E020EEA2252
:100C5000EF50460802E108D004D029C2E6FF34DF95
:100C6000E5520201282BE0D72851EA6A2A0FE96EE3
:100C7000020EEA22EF6A12000201286B070E285DBD
:100C800016E22851EA6A2A0FE96E020EEA22EF50B4
:100C9000E66E1ADFE55202012829EA6A2A0FE96E98
:100CA000020EEA22EF5001E102D0282BE7D7120012
:100CB0000F0EC16E936A3C0E926E0F0E946E80A85A
:100CC00022D0010E816E0201336B346B080E34AFFB
:100CD00002D0D89003D0335D000E345913E28070F7
:100CE000C80EE66EE66AE66AE66AA6DDE552E552F9
:100CF000E552E5528150E824816E0201332B000E4B
:080D00003423E4D7DCD7120014
:080D08002A0EF66E080EF76ECC
:100D1000000EF86E02010900F5503A6F0900F55017
:100D20003B6F03E13A6701D03DD00900F550356FC4
:100D30000900F550366F0900F550376F09000900BA
:100D4000F550E96E0900F550EA6E09000900090046
:100D5000F550386F0900F550396F09000900F6CFDA
:100D60003CF2F7CF3DF2F8CF3EF235C2F6FF36C285
:100D7000F7FF37C2F8FF0201385302E1395307E0A9
:100D80000900F550EE6E3807F8E23907F9D73CC292
:100D9000F6FF3DC2F7FF3EC2F8FF02013A07000E20
:060DA0003B5BBFD712000F
:0A0DA600FF0EE350066E480E01D068
:100DB0004C0EE76EE72EFED7E76AE72EFED7062E2B
:060DC000F7D7000012004D
:0A0DC600000EF36E00EE00F0080EC0
:100DD00001D81200EA6002D0EE6AFCD7F350E96055
:060DE0001200EE6AFCD7D0
:0A0DE60012EE40F022EE40F0F86A31
:100DF000059C84EC06F001EC07F058EC06F0FBD7FC
:020E00001200DE
:020E02001200DC
:0C0E0400EEEDEBE7DEDDDBD7BEBDBBB7DB
:100E10007E7D7B7730313233343536373839414255
:040E200043444546BC
:00000001FF
